BL51 BANKED LINKER/LOCATER V6.22                                                        09/28/2022  19:51:28  PAGE 1


BL51 BANKED LINKER/LOCATER V6.22, INVOKED BY:
C:\KEIL_V4\C51\BIN\BL51.EXE .\Release\system_FE81001.obj, .\Release\STARTUP.obj, .\Release\main.obj TO .\Release\Sample_
>> DrvI2C_Master REGFILE (.\Release\Sample_DrvI2C_Master.ORC) PRINT (.\Sample_DrvI2C_Master.m51) RAMSIZE (256) CODE (0X0
>> 000-0X1FFF) XDATA (0X8000-0X87FF)


MEMORY MODEL: SMALL


INPUT MODULES INCLUDED:
  .\Release\system_FE81001.obj (SYSTEM_FE81001)
  .\Release\STARTUP.obj (?C_STARTUP)
  .\Release\main.obj (MAIN)
  C:\KEIL_V4\C51\LIB\C51S.LIB (?C_INIT)
  C:\KEIL_V4\C51\LIB\C51S.LIB (?C?CLDOPTR)
  C:\KEIL_V4\C51\LIB\C51S.LIB (?C_IBP)


LINK MAP OF MODULE:  .\Release\Sample_DrvI2C_Master (SYSTEM_FE81001)


            TYPE    BASE      LENGTH    RELOCATION   SEGMENT NAME
            -----------------------------------------------------

            * * * * * * *   D A T A   M E M O R Y   * * * * * * *
            REG     0000H     0008H     ABSOLUTE     "REG BANK 0"
            DATA    0008H     0015H     UNIT         ?DT?MAIN
            DATA    001DH     0007H     UNIT         ?DT?_I2C_MASTER_READ?MAIN
            DATA    0024H     0006H     UNIT         ?DT?_DELAY?MAIN
            DATA    002AH     0006H     UNIT         ?DT?_I2C_MASTER_WRITE?MAIN
            DATA    0030H     0002H     UNIT         ?DT?I2CISR?MAIN
            DATA    0032H     0001H     UNIT         ?C?LIB_DATA
            IDATA   0033H     0001H     UNIT         ?STACK

            * * * * * * *   C O D E   M E M O R Y   * * * * * * *
            CODE    0000H     0003H     ABSOLUTE     
            CODE    0003H     003BH     UNIT         ?PR?_DELAY?MAIN
            CODE    003EH     001CH     UNIT         ?C_INITSEG
            CODE    005AH     0001H     UNIT         ?PR?SYSTEMINIT?SYSTEM_FE81001
            CODE    005BH     0003H     ABSOLUTE     
            CODE    005EH     0176H     UNIT         ?PR?_I2C_MASTER_READ?MAIN
            CODE    01D4H     00C0H     UNIT         ?PR?_I2C_MASTER_WRITE?MAIN
            CODE    0294H     009DH     UNIT         ?C_C51STARTUP
            CODE    0331H     0090H     UNIT         ?PR?IOCONFIG?MAIN
            CODE    03C1H     0079H     UNIT         ?PR?MAIN?MAIN
            CODE    043AH     0059H     UNIT         ?PR?I2CISR?MAIN
            CODE    0493H     002DH     UNIT         ?C?LIB_CODE
            CODE    04C0H     0017H     UNIT         ?PR?CLKCONFIG?MAIN
            CODE    04D7H     0017H     UNIT         ?PR?I2C_MASTER_CONFIG?MAIN



OVERLAY MAP OF MODULE:   .\Release\Sample_DrvI2C_Master (SYSTEM_FE81001)


SEGMENT
  +--> CALLED SEGMENT
---------------------
BL51 BANKED LINKER/LOCATER V6.22                                                      09/28/2022  19:51:28  PAGE 2


?C_C51STARTUP
  +--> ?PR?MAIN?MAIN
  +--> ?C_INITSEG

?PR?MAIN?MAIN
  +--> ?PR?I2C_MASTER_CONFIG?MAIN
  +--> ?PR?_I2C_MASTER_WRITE?MAIN
  +--> ?PR?_I2C_MASTER_READ?MAIN

?PR?I2C_MASTER_CONFIG?MAIN
  +--> ?PR?CLKCONFIG?MAIN
  +--> ?PR?IOCONFIG?MAIN



SYMBOL TABLE OF MODULE:  .\Release\Sample_DrvI2C_Master (SYSTEM_FE81001)

  VALUE           TYPE          NAME
  ----------------------------------

  -------         MODULE        SYSTEM_FE81001
  C:0000H         SYMBOL        _ICE_DUMMY_
  C:005AH         PUBLIC        SystemInit
  -------         PROC          SYSTEMINIT
  C:005AH         LINE#         38
  C:005AH         LINE#         39
  C:005AH         LINE#         41
  -------         ENDPROC       SYSTEMINIT
  -------         ENDMOD        SYSTEM_FE81001

  -------         MODULE        ?C_STARTUP
  C:0294H         SEGMENT       ?C_C51STARTUP
  I:0033H         SEGMENT       ?STACK
  C:0000H         PUBLIC        ?C_STARTUP
  D:00E0H         SYMBOL        ACC
  D:00F0H         SYMBOL        B
  D:0083H         SYMBOL        DPH
  D:0082H         SYMBOL        DPL
  N:0001H         SYMBOL        IBPSTACK
  N:0100H         SYMBOL        IBPSTACKTOP
  N:0080H         SYMBOL        IDATALEN
  C:0297H         SYMBOL        IDATALOOP
  N:0000H         SYMBOL        PBPSTACK
  N:0100H         SYMBOL        PBPSTACKTOP
  N:0000H         SYMBOL        PDATALEN
  N:0000H         SYMBOL        PDATASTART
  N:0000H         SYMBOL        PPAGE
  N:0000H         SYMBOL        PPAGEENABLE
  D:00A0H         SYMBOL        PPAGE_SFR
  D:0081H         SYMBOL        SP
  C:0294H         SYMBOL        STARTUP1
  N:0000H         SYMBOL        XBPSTACK
  N:0000H         SYMBOL        XBPSTACKTOP
  N:0800H         SYMBOL        XDATALEN
  C:02A2H         SYMBOL        XDATALOOP
  N:8000H         SYMBOL        XDATASTART
  C:0000H         LINE#         126
BL51 BANKED LINKER/LOCATER V6.22                                                      09/28/2022  19:51:28  PAGE 3


  C:0294H         LINE#         133
  C:0296H         LINE#         134
  C:0297H         LINE#         135
  C:0298H         LINE#         136
  C:029AH         LINE#         140
  C:029DH         LINE#         141
  C:029FH         LINE#         145
  C:02A1H         LINE#         147
  C:02A2H         LINE#         148
  C:02A3H         LINE#         149
  C:02A4H         LINE#         150
  C:02A6H         LINE#         151
  C:02A8H         LINE#         170
  C:02ABH         LINE#         185
  C:02AEH         LINE#         196
  -------         ENDMOD        ?C_STARTUP

  -------         MODULE        MAIN
  C:0000H         SYMBOL        _ICE_DUMMY_
  D:0090H         PUBLIC        P1
  D:00B0H         PUBLIC        P3
  D:0008H         PUBLIC        I2C_RX_Buffer
  D:0012H         PUBLIC        I2C_TX_Buffer
  D:00A8H         PUBLIC        IE
  C:0003H         PUBLIC        _delay
  D:00B8H         PUBLIC        IP
  C:03C1H         PUBLIC        main
  C:043AH         PUBLIC        I2CISR
  D:0098H         PUBLIC        SCON
  C:04C0H         PUBLIC        CLKConfig
  D:0088H         PUBLIC        TCON
  D:001CH         PUBLIC        cnt
  C:04D7H         PUBLIC        I2C_Master_Config
  D:00C8H         PUBLIC        T2CON
  C:005EH         PUBLIC        _I2C_Master_Read
  C:0331H         PUBLIC        IOConfig
  D:00D0H         PUBLIC        PSW
  C:01D4H         PUBLIC        _I2C_Master_Write
  -------         PROC          _DELAY
  D:0024H         SYMBOL        cnt
  -------         DO            
  D:0026H         SYMBOL        i
  D:0028H         SYMBOL        j
  -------         ENDDO         
  C:0003H         LINE#         38
  C:0007H         LINE#         39
  C:0007H         LINE#         42
  C:0018H         LINE#         43
  C:003DH         LINE#         45
  -------         ENDPROC       _DELAY
  -------         PROC          I2CISR
  -------         DO            
  D:0030H         SYMBOL        int_stat
  -------         ENDDO         
  C:043AH         LINE#         58
  C:044DH         LINE#         62
  C:0467H         LINE#         66
BL51 BANKED LINKER/LOCATER V6.22                                                      09/28/2022  19:51:28  PAGE 4


  C:046CH         LINE#         67
  C:046CH         LINE#         70
  C:0471H         LINE#         71
  C:047CH         LINE#         73
  C:047CH         LINE#         76
  C:047CH         LINE#         77
  C:047CH         LINE#         80
  C:0482H         LINE#         81
  -------         ENDPROC       I2CISR
  -------         PROC          IOCONFIG
  C:0331H         LINE#         93
  C:0331H         LINE#         94
  C:0331H         LINE#         96
  C:0352H         LINE#         100
  C:0368H         LINE#         101
  C:037EH         LINE#         104
  C:039FH         LINE#         107
  C:03C0H         LINE#         108
  -------         ENDPROC       IOCONFIG
  -------         PROC          CLKCONFIG
  C:04C0H         LINE#         120
  C:04C0H         LINE#         121
  C:04C0H         LINE#         123
  C:04CBH         LINE#         126
  C:04D6H         LINE#         128
  -------         ENDPROC       CLKCONFIG
  -------         PROC          _I2C_MASTER_WRITE
  D:002AH         SYMBOL        data_
  D:002DH         SYMBOL        len
  D:002EH         SYMBOL        slave_address
  -------         DO            
  D:002FH         SYMBOL        i
  -------         ENDDO         
  C:01D4H         LINE#         142
  C:01DCH         LINE#         143
  C:01DCH         LINE#         146
  C:01E2H         LINE#         149
  C:01E8H         LINE#         152
  C:01EEH         LINE#         153
  C:01F3H         LINE#         156
  C:01F8H         LINE#         157
  C:01FDH         LINE#         161
  C:0203H         LINE#         162
  C:0209H         LINE#         163
  C:0212H         LINE#         164
  C:0218H         LINE#         167
  C:021EH         LINE#         168
  C:0224H         LINE#         169
  C:022DH         LINE#         170
  C:0233H         LINE#         173
  C:023DH         LINE#         174
  C:023DH         LINE#         175
  C:0243H         LINE#         176
  C:0249H         LINE#         177
  C:025FH         LINE#         178
  C:0265H         LINE#         179
  C:026EH         LINE#         180
BL51 BANKED LINKER/LOCATER V6.22                                                      09/28/2022  19:51:28  PAGE 5


  C:0274H         LINE#         181
  C:0278H         LINE#         184
  C:027EH         LINE#         185
  C:0284H         LINE#         186
  C:028DH         LINE#         187
  C:0293H         LINE#         189
  -------         ENDPROC       _I2C_MASTER_WRITE
  -------         PROC          _I2C_MASTER_READ
  D:001DH         SYMBOL        data_
  D:0020H         SYMBOL        len_W
  D:0021H         SYMBOL        len_R
  D:0022H         SYMBOL        slave_address
  -------         DO            
  D:0023H         SYMBOL        i
  -------         ENDDO         
  C:005EH         LINE#         204
  C:0066H         LINE#         205
  C:0066H         LINE#         210
  C:006CH         LINE#         213
  C:0072H         LINE#         216
  C:0078H         LINE#         217
  C:007DH         LINE#         220
  C:0082H         LINE#         221
  C:0087H         LINE#         225
  C:008DH         LINE#         226
  C:0093H         LINE#         227
  C:009CH         LINE#         228
  C:00A2H         LINE#         231
  C:00A8H         LINE#         232
  C:00AEH         LINE#         233
  C:00B7H         LINE#         234
  C:00BDH         LINE#         238
  C:00C7H         LINE#         239
  C:00C7H         LINE#         240
  C:00CDH         LINE#         241
  C:00D3H         LINE#         242
  C:00D9H         LINE#         244
  C:00EFH         LINE#         245
  C:00F5H         LINE#         246
  C:00FEH         LINE#         247
  C:0104H         LINE#         248
  C:0108H         LINE#         252
  C:010EH         LINE#         255
  C:0114H         LINE#         258
  C:011AH         LINE#         261
  C:0120H         LINE#         262
  C:0125H         LINE#         265
  C:012BH         LINE#         266
  C:0131H         LINE#         267
  C:013AH         LINE#         268
  C:0140H         LINE#         271
  C:0146H         LINE#         272
  C:014CH         LINE#         273
  C:0155H         LINE#         274
  C:015BH         LINE#         276
  C:0161H         LINE#         277
  C:0167H         LINE#         278
BL51 BANKED LINKER/LOCATER V6.22                                                      09/28/2022  19:51:28  PAGE 6


  C:016DH         LINE#         280
  C:0177H         LINE#         282
  C:0180H         LINE#         283
  C:018BH         LINE#         285
  C:0191H         LINE#         287
  C:0199H         LINE#         288
  C:0199H         LINE#         289
  C:019FH         LINE#         290
  C:01A1H         LINE#         292
  C:01A1H         LINE#         293
  C:01A7H         LINE#         294
  C:01A7H         LINE#         296
  C:01B4H         LINE#         298
  C:01B8H         LINE#         301
  C:01BEH         LINE#         302
  C:01C4H         LINE#         303
  C:01CDH         LINE#         304
  C:01D3H         LINE#         306
  -------         ENDPROC       _I2C_MASTER_READ
  -------         PROC          I2C_MASTER_CONFIG
  C:04D7H         LINE#         308
  C:04D7H         LINE#         309
  C:04D7H         LINE#         310
  C:04DAH         LINE#         311
  C:04DDH         LINE#         312
  C:04EDH         LINE#         314
  -------         ENDPROC       I2C_MASTER_CONFIG
  -------         PROC          MAIN
  C:03C1H         LINE#         325
  C:03C1H         LINE#         326
  C:03C1H         LINE#         327
  C:03C4H         LINE#         329
  C:03CAH         LINE#         330
  C:03D0H         LINE#         331
  C:03D6H         LINE#         334
  C:03D9H         LINE#         335
  C:03DCH         LINE#         336
  C:03DFH         LINE#         337
  C:03EDH         LINE#         340
  C:03F0H         LINE#         341
  C:0401H         LINE#         345
  C:0401H         LINE#         347
  C:0401H         LINE#         348
  C:0414H         LINE#         349
  C:0414H         LINE#         350
  C:0419H         LINE#         351
  C:041EH         LINE#         352
  C:0423H         LINE#         354
  C:0425H         LINE#         356
  C:0425H         LINE#         357
  C:042BH         LINE#         358
  C:0431H         LINE#         359
  C:0437H         LINE#         360
  C:0437H         LINE#         362
  C:0439H         LINE#         363
  -------         ENDPROC       MAIN
  -------         ENDMOD        MAIN
BL51 BANKED LINKER/LOCATER V6.22                                                      09/28/2022  19:51:28  PAGE 7



  -------         MODULE        ?C?CLDOPTR
  C:0493H         PUBLIC        ?C?CLDOPTR
  -------         ENDMOD        ?C?CLDOPTR

  -------         MODULE        ?C_IBP
  D:0032H         PUBLIC        ?C_IBP
  -------         ENDMOD        ?C_IBP



FUNCTION REGISTER MASKS


FUNCTION . . . . . . . . . REG MASK
-----------------------------------

CLKCONFIG. . . . . . . . . @0xe301
I2CISR . . . . . . . . . . @0xe30f
I2C_MASTER_CONFIG. . . . . @0xe301
IOCONFIG . . . . . . . . . @0xe301
MAIN . . . . . . . . . . . @0xf3f7
SYSTEMINIT . . . . . . . . @0x8000
_DELAY . . . . . . . . . . @0xf000
_I2C_MASTER_READ . . . . . @0xf3f3
_I2C_MASTER_WRITE. . . . . @0xf3f1

*** WARNING L16: UNCALLED SEGMENT, IGNORED FOR OVERLAY PROCESS
    SEGMENT: ?PR?SYSTEMINIT?SYSTEM_FE81001

*** WARNING L16: UNCALLED SEGMENT, IGNORED FOR OVERLAY PROCESS
    SEGMENT: ?PR?_DELAY?MAIN

Program Size: data=52.0 xdata=0 code=1262
LINK/LOCATE RUN COMPLETE.  2 WARNING(S),  0 ERROR(S)
